:020000040000FA
:100000000608A20083169B0183129F0183169F019D
:1000100007309C008F300F0570388F005428A601E0
:10002000A7012428831203130330A0008330A1000A
:100030000A128A11A10B18280A128A11A00B16287D
:100040008316A60A0319A70A260824028312A00011
:1000500083162708250283122004031D1228080096
:10006000A201A301482883120313B430A000DD309D
:10007000A1000A128A11A10B39280A128A11A00BB9
:1000800037280000000000008316A20A0319A30A03
:10009000220820028312A000831623082102831263
:1000A0002004031D33280800473081008610061104
:1000B0008611061286120613861306148312241064
:1000C000A301152CA30124186D10241C6D140530F8
:1000D0002302ED1003196E28031CED146D156D1825
:1000E000ED1C6D116D1D9128FF30EE006E08A20011
:1000F000220886000618241401308316A000A101EE
:100100003020831206182414EF016F08A200220881
:10011000860001308316A000A10130208312A30ABB
:10012000632808000A308316A000A1013020831242
:1001300006182414FB30E7006708A2002208860096
:1001400001308316A000A1013020F0308312E800B6
:100150006808A2002208860001308316A000A101D1
:100160003020E0308312E9006908A20022088600EE
:1001700001308316A000A1013020C0308312EA00B4
:100180006A08A2002208860001308316A000A1019F
:10019000302080308312EB006B08A200220886001A
:1001A00001308316A000A10130208312EC016C08FD
:1001B000A2002208860001308316A000A101302091
:1001C0008312061824140800A30124184F10241CBD
:1001D0004F1402302302CF100319F028031CCF1450
:1001E0004F154F18CF1C4F114F1D0D2AD10151082B
:1001F000A2002208860001308316A000A101302051
:1002000004308312D2005208A20022088600013076
:100210008316A000A10130200B308312D3005308B5
:10022000A2002208860001308316A000A101302020
:1002300010308312D4005408A20022088600013036
:100240008316A000A101302020308312D50055086C
:10025000A2002208860001308316A000A1013020F0
:1002600040308312D6005608A200220886000130D2
:100270008316A000A101302080308312D7005708D8
:10028000A2002208860002308316A000A1013020BF
:100290008312061824148430D8005808A2002208BB
:1002A000860001308316A000A10130208B3083121C
:1002B000D9005908A2002208860001308316A00048
:1002C000A101302090308312DA005A08A2002208DF
:1002D000860001308316A000A1013020A0308312D7
:1002E000DB005B08A2002208860001308316A00014
:1002F000A1013020C0308312DC005C08A20022087B
:10030000860002308316A000A10130208312061857
:100310002414C430DD005D08A200220886000130EC
:100320008316A000A1013020CB308312DE005E08CE
:10033000A2002208860001308316A000A10130200F
:10034000D0308312DF005F08A2002208860001304F
:100350008316A000A1013020E0308312E000600885
:10036000A2002208860002308316A000A1013020DE
:10037000831206182414E430E1006108A200220868
:10038000860001308316A000A1013020EB308312DB
:10039000E2006208A2002208860001308316A00055
:1003A000A1013020F0308312E3006308A20022088C
:1003B000860002308316A000A101302083120618A7
:1003C0002414F430E4006408A200220886000130FE
:1003D0008316A000A1013020FB308312E5006508E0
:1003E000A2002208860002308316A000A10130205E
:1003F000831206182414FF30E6006608A2002208C3
:10040000860002308316A000A10130208312061856
:10041000241492208312A30AE5280800A3012418BB
:100420003710241C371405302302B71003191A2A79
:10043000031CB71437153718B71C3711371D9E2A00
:100440008030B9003908A2002208860001308316E6
:10045000A000A101302040308312BA003A08A20067
:100460002208860001308316A000A1013020203030
:100470008312BB003B08A2002208860001308316CD
:10048000A000A101302010308312BC003C08A20063
:100490002208860001308316A000A10130200B3015
:1004A0008312BD003D08A200220886000130831699
:1004B000A000A101302004308312BE003E08A2003B
:1004C000220886000618241401308316A000A1011A
:1004D00030200B308312BF003F08A20022088600A4
:1004E00001308316A000A101302010308312C0001B
:1004F0004008A2002208860001308316A000A10156
:10050000302020308312C1004108A200220886005A
:1005100001308316A000A101302040308312C200B8
:100520004208A2002208860001308316A000A10123
:100530003020831206182414A30A0F2AA3012418BA
:10054000B712241CB7160530230237130319AA2A41
:10055000031C3717B717B71A371FB713B71F442B2A
:100560008030C3004308A2002208860001308316B1
:10057000A000A1013020C0308312C4004408A200B2
:100580002208860001308316A000A1013020E0304F
:100590008312C5004508A200220886000130831698
:1005A000A000A1013020F0308312C6004608A2004E
:1005B0002208860001308316A000A1013020FB3004
:1005C0008312C7004708A200220886000130831664
:1005D000A000A1013020FF308312C8004808A2000B
:1005E0002208860002308316A000A10130207F304F
:1005F0008312C9004908A200220886000130831630
:10060000A000A10130203F308312CA004A08A20096
:100610002208860001308316A000A10130201F307F
:100620008312CB004B08A2002208860001308316FB
:10063000A000A10130200F308312CC004C08A20092
:100640002208860001308316A000A101302004306A
:100650008312CD004D08A2002208860001308316C7
:10066000A000A10130208312CE014E08A200220872
:10067000860002308316A000A10130208312A30A55
:10068000061C9F2A24149F2A08003230A900B001BA
:100690003008A20022088600AA01A21722088600BC
:1006A00001308316A400A5010F208312A213220893
:1006B000860029088316A400A5010F208312A90330
:1006C000AA0A32302A02031D4D2B8030B1003108B6
:1006D000A200220886003230A900AB0122172208AE
:1006E000860001308316A400A5010F208312221377
:1006F0002208860029088316A400A5010F20831272
:10070000A903AB0A32302B02031D6E2BC030B2009E
:100710003208A200220886003230A900AC01A216DD
:100720002208860001308316A400A5010F20831241
:10073000A2122208860029088316A400A5010F2012
:100740008312A903AC0A32302C02031D8F2BE03038
:10075000B3003308A200220886003230A900AD01A0
:1007600022162208860001308316A400A5010F205E
:10077000831222122208860029088316A400A501EC
:100780000F208312A903AD0A32302D02031DB02BB6
:10079000F030B4003408A200220886003230A900EC
:1007A000AE01A2152208860001308316A400A5011F
:1007B0000F208312A2112208860029088316A400A4
:1007C000A5010F208312A903AE0A32302E02031DA9
:1007D000D12BFB30B5003508A2002208860032304C
:1007E000A900AF0122152208860001308316A4005B
:1007F000A5010F20831222112208860029088316E2
:10080000A400A5010F208312A903AF0A32302F02E2
:10081000031DF22BFF30B6003608A2002208860026
:100820000A308316A000A1013028241C6220831204
:10083000241CE4208312241C0E228312241C452332
:100840008312241C152C2410A5012508A2002208BF
:1008500086008B108B130B16630000008B1C152C6D
:10086000A6015430A7002708A200220886003230D3
:100870008316A400A5010F20A8308312A800280821
:10088000A2002208860032308316A400A5010F20A2
:0E0890008312A60A0A302602031D312C152CF5
:02400E00783FF9
:02401000FF3F70
:00000001FF
